:1000000000308A000428000084011F30830571300D
:1000100083168F0083121F1383161F109F101F114A
:100020009F110730831299003B308316850083129D
:100030001F1383161F149F101F119F111F129F164D
:100040001F1383129F171F1407309900831605088A
:1000500006308312A000A00B2B28000019088C1179
:1000600083160511831205110C3095000030A10094
:1000700005389200FF308316920071308F00C03037
:1000800083128B040030A1001F08F33921049F0064
:100090000630A000A00B4A2800009F149F184E288D
:1000A00083161E088312A6001E08A7002708A200B8
:1000B0002608A100A20CA10CA20CA10CA20C2108E4
:1000C0009300A20C220C3039A0001508CF3920046F
:0600D000950042286300C8
:02400E00C43FAD
:00000001FF
